:1000000012C01895189518956CC6189518951895DE
:100010001895189518951895189518951895189578
:100020001895189518958FE58DBFC0E2E8EF4E2E14
:1000300084E08EBFD4E0F3E05F2EEEEFF3E0A0E6C5
:10004000B0E088278D933197E9F78CE089B980E09B
:1000500080BD88E18AB9FDD36624FBD388E082BDE8
:1000600085E085BD89B7806489BF789480E087BBCF
:10007000C09AC19AECE8F0E080E433D458E0C89527
:10008000802D29D431965A95D1F704C00609090666
:1000900020202020ECEAF0E088E423D458E0C89542
:1000A000802D19D431965A95D1F704C00101010170
:1000B00020202020ECECF0E080E513D458E0C89537
:1000C000802D09D431965A95D1F704C020202020E4
:1000D00010101010ECEEF0E088E503D458E0C8955D
:1000E000802DF9D331965A95D1F704C00204081037
:1000F00020202020ECE0F1E080E6F3D358E0C89522
:10010000802DE9D331965A95D1F704C020202001E3
:1001100002040810ECE2F1E088E6E3D358E0C89569
:10012000802DD9D331965A95D1F704C02020201FB5
:1001300020202020ECE4F1E080E7D3D358E0C895FC
:10014000802DC9D331965A95D1F704C00804020115
:1001500020202020ECE6F1E088E7C3D358E0C895E2
:10016000802DB9D331965A95D1F704C020202010A4
:10017000080402018EE1809361008CE080936200AC
:100180004ED38CE0AED3E4E8FEE043D38FEB11E036
:1001900055D3E6E9FEE03DD3E1E0F0E051D33FD3B3
:1001A00080E0E3E3F4D4AFE7B0E0EEE9F0E098E01C
:1001B00054D680E0E3E3F0D4A7E8B0E0EEE9F0E065
:1001C00098E04BD6002762FA0EF401E041E00417F4
:1001D00009F0EFCF80E0E3E34FD5A8E7B0E00C9360
:1001E00087E0EFE7F0E03ED6402F0091860004174D
:1001F00009F018C08FE711E021D300917F00083289
:1002000009F004C0E8EAFEE004D30CC000917F00CE
:10021000003109F004C0EAEBFEE0FBD203C0ECECD5
:10022000FEE0F7D287E0E7E8F0E01CD6402F00912F
:100230008E00041709F021C08FEB11E0FFD200916E
:100240007800013009F004C0EEEDFEE0E2D215C006
:1002500000918700083209F004C0E0EFFEE0D9D237
:100260000CC000918700003109F004C0E2E0FFE01B
:10027000D0D203C0E4E1FFE0CCD2E2E0F0E0E0D293
:10028000CED2A0E9B0E08C918F5F8C930027A6E3DB
:10029000B0E08C9180FB0EF401E040E0041709F01F
:1002A00001C073D10027A6E3B0E08C9181FB0EF46E
:1002B00001E040E0041709F001C077D186D1EF9347
:1002C000FF93E4ECF0E02DD3FF91EF91EF93FF93D8
:1002D000E4ECF0E026D3FF91EF91EF93FF93E4EC91
:1002E000F0E01FD3FF91EF91EF93FF93E4ECF0E088
:1002F00018D3FF91EF918FE711E0A0D2E6E2FFE083
:1003000088D202E081D2EAE2FFE083D2009162006B
:100310000A3008F00AC0ECE2FFE07BD2A0EEB3E0C6
:10032000E2E6F0E04FD568D206C0A0EEB3E0E2E628
:10033000F0E048D561D2EEE2FFE06BD20091900090
:10034000043010F009F001C003C081E080939000F8
:10035000009161000A3008F00AC0ECE2FFE059D2D7
:10036000A0EEB3E0E1E6F0E02DD546D206C0A0EE67
:10037000B3E0E1E6F0E026D53FD2E0E3FFE049D28A
:1003800080E0E3E3AFE7B0E08AD48FEB11E056D230
:10039000002762FA0EF401E041E0041709F004C0FE
:1003A000E6E3FFE036D25AC06EEB80E0E3E3BB2722
:1003B000A6E121E02A9368D380E0A1E9B0E0E3E37D
:1003C00029E02A938BD388E0E1E9F0E04BD5402F78
:1003D00000919900041709F041C000917F0000319D
:1003E00009F012C0E9E7F0E0FA93EA935A924A92D0
:1003F00080919900A42DB52D8C9381E0BAD13BD189
:10040000249681E0B2D116C000917F00083209F035
:1004100011C0E9E7F0E0FA93EA935A924A92809188
:100420009900A42DB52D8C9381E0A3D1E2D0249620
:1004300081E09BD1ABE7B0E0E9E7F0E0BCD4EBE7CB
:10044000F0E0A0EEB3E0112721E003E031E0A2D21A
:10045000D3D180E040D2EEE3FFE0DBD10091900009
:10046000013009F005C081E036D282E034D217C0F5
:10047000023009F005C084E02ED283E02CD20FC0F8
:10048000033009F005C085E026D285E024D207C0FC
:10049000043009F004C086E01ED287E01CD280E060
:1004A000E3E3A7E8B0E0FBD38FEB1AE0C7D1002766
:1004B00062FA0EF401E041E0041709F004C0E0E440
:1004C000FFE0A7D15AC06EEB80E0E3E3BB27A6E1D3
:1004D00021E02A93D9D280E0A1E9B0E0E3E329E06A
:1004E0002A93FCD288E0E1E9F0E0BCD4402F0091EF
:1004F0009900041709F041C000918700003109F00C
:1005000012C0E9E7F0E0FA93EA935A924A92809196
:100510009900A42DB52D8C9381E02BD1ACD02496DD
:1005200081E023D116C000918700083209F011C084
:10053000E9E7F0E0FA93EA935A924A92809199009F
:10054000A42DB52D8C9381E014D153D0249681E055
:100550000CD1ABE7B0E0E9E7F0E02DD4EBE7F0E059
:10056000A0EEB3E0112721E003E031E013D244D143
:1005700080E0B1D1EEE3FFE04CD101E045D184EF62
:1005800091E0DBD17ECEF894FFCFA1E6B0E08C9174
:100590008F5F8C93009161000B3310F009F001C064
:1005A00003C080E0809361000895A2E6B0E08C91E2
:1005B0008F5F8C9300916200073110F009F001C049
:1005C00003C080E080936200089580E0E3E330D2CE
:1005D0006CEC80E0E3E3BB27A6E121E02A9354D250
:1005E00064E480E0E3E3BB27A6E121E02A934CD258
:1005F000089580E090E0AA81BB818D939C93A2E94D
:10060000B0E09C91A1E9B0E08C91AA81BB818D936F
:100610009C93A2E9B0E00C9107FB00270EF401E0E7
:1006200041E0041709F010C0AA81BB8142E095D0D7
:10063000AA81BB810D911C9141E050E0040F151F70
:10064000AA81BB810D931C93AA81BB810D911C9142
:100650004AE050E081D1AA81BB810D931C93AA810D
:10066000BB810D911C9140E150E08CD0AA81BB81EF
:100670004D935C9308950091910041E00423A6EA14
:10068000B0E00C930091A600013009F005C0809104
:100690009100815080939100A2E9B0E09C91A1E982
:1006A000B0E08C91A7EAB0E08D939C93A7EAB0E00C
:1006B0000D911C9142E350E04FD1A7EAB0E00D93B9
:1006C0001C93A7EAB0E00D911C9149E150E0041B96
:1006D000150BA7EAB0E00D931C93A8E9B0E00D91CB
:1006E0001127A7E9B0E04D915527041B150BA9EA86
:1006F000B0E00D931C93A9EAB0E00D911C9144E683
:1007000050E02AD1A9EAB0E00D931C93A9EAB0E029
:100710000D911C91A8E9B0E04D91552733D0A9EA7D
:10072000B0E04D935C93A7EAB0E00D911C91A9EA6B
:10073000B0E04D915C91040F151FA7EAB0E00D9356
:100740001C93A7EAB0E00D911C914AE050E01AD04A
:10075000AA81BB814D935C930895EA2FFB2F8D9165
:10076000809581934A95D9F70895481A8827580AA1
:100770000895480E8827581E089508D0EDD000FC33
:1007800010D0089503D01ED001F8F9CF0024E894CA
:1007900057FF02C009D0689400F80BD010F801246C
:1007A000089502D009D00895509540954F5F5F4F4E
:1007B0000895E89417FF0895009510950F5F1F4F57
:1007C00068940895352F242FE894452B11F46894EC
:1007D0000895512F402F0027112780E1440F551F06
:1007E000001F111F021B130B416018F4020F131F8F
:1007F0004E7F8A9599F70895A0EEB3E08D918823F6
:1008000011F069D0FBCF089580E265D00A95E1F739
:100810000895ACD0802D11F05ED0FBCF089581E01B
:1008200060D014D080E85DC08FE7213039F08FEBC5
:10083000223021F08FE8233009F08FEC810F51C076
:1008400088EE93E07AD03197D9F7089583E099271D
:1008500074C08AEF90E071D08F9A8E9A8D9A8C9A9C
:100860008A9A8B9A939885E090E067D092989798AF
:100870009698959A949A929AEF93FF93E0E6F0E017
:1008800050D0FF91EF91929855D0929AEF93FF93A9
:10089000E0E6F0E046D0FF91EF9192984BD0929A2B
:1008A000EF93FF93E0E6F0E03CD0FF91EF91929858
:1008B00041D09498929AEF93FF93E0E6F0E031D024
:1008C000FF91EF91929836D088E20BD08EE009D05C
:1008D00086E007D00895939A829505D004D02AD057
:1008E00008959398F9CF859510F4949A01C094983F
:1008F000859510F4959A01C09598859510F4969A6F
:1009000001C09698859510F4979A01C09798929A8D
:10091000EF93FF93E0E6F0E004D0FF91EF9192981F
:1009200008953197F1F70895689462F80895E8946E
:1009300062F8089581E090E000C0EF93FF93EE2706
:10094000E82BE92B31F0E8EEF3E03197F1F701976E
:10095000D1F7FF91EF9108950F92B801469F800162
:10096000479F100D569F100D0F900895C895319612
:100970000020089591E0882321F08894991F8A959A
:10098000E9F7892F90950895883018F011968850CE
:10099000FBCF08952E2E3F2E992781918D3209F09D
:1009A00093958823D1F79A95E22DF32D112361F0C9
:1009B000091718F011F0101B01C0191B28F021F0C5
:1009C00080E28D931A95E9F780818D3219F48D9329
:1009D000319604C0222311F08BE28D93091738F071
:1009E00031F0091B21F080E38D930A95E9F781919D
:1009F0008D938823E1F7332351F0EA2FFB2F3196B3
:100A000033958E9182933A95E1F78EE28C93089517
:100A10000181082B01831281192312830000000039
:100A20000000000000000000000000000000089529
:100A30007BDFFF279FDFECDFEF93FF93ECEDF1E02F
:100A400070DFFF91EF91182B128309230183EF933D
:100A5000FF93E6E5F0E065DFFF91EF911081182349
:100A600059F4EF93FF93ECEDF1E05BDFFF91EF9131
:100A70001081182309F05BDFEF93FF93ECEDF1E0B9
:100A800050DFFF91EF91089575DFFF2729915D9168
:100A900048E0BEDF00000000000000000000000091
:100AA000000000000000579510F4182B1283EF93FC
:100AB000FF93E8E3F0E035DFFF91EF91182B12830D
:100AC0000000000000000000000000000000000026
:100AD00000004A95F1F62A95D1F608954BDFFF27DD
:100AE000299148E0552794DF09230183EF93FF9371
:100AF000E2E0F0E016DFFF91EF9188941081182377
:100B000009F008945795EF93FF93E9E2F0E009DFCD
:100B1000FF91EF914A9539F75D932A9511F7089562
:100B200077DF09230183EF93FF93E2E0F0E0F9DE42
:100B3000FF91EF91E8941081182309F06894EF93E6
:100B4000FF93EEE2F0E0EDDEFF91EF91089560DFBC
:100B50000000000000000000000000000000000095
:100B6000000016F4182B1283EF93FF93E8E3F0E0F4
:100B7000D8DEFF91EF91182B1283000000000000D7
:100B8000000000000000000000000000089533276E
:100B900030939D0030939A004BDF0EF458C0309193
:100BA0009A0030FD54C0662760939C006395609363
:100BB0009B0021E050EF48E06CDFB2DF31F9B0DF9D
:100BC00032F9632F6670663009F441C0603019F065
:100BD00031FB40D025C060919B0070919D0067174C
:100BE000B1F0C0F48F939F93862F8A95AEE9B0E061
:100BF000CBDEC0DE7C9178236894772329F4E894D7
:100C000060919B0060939C009F918F9109C06894B4
:100C100021D006C0E8941ED060919B0060939C0098
:100C200096DF60919B00639560939B00613409F0AF
:100C3000C4CF60919C0060939D006623E89409F402
:100C4000689430F930939A00E89462F808956894B3
:100C500062F808958F939F93AEE9B0E080919B0076
:100C60008A9592DE87DE7C9116F4782B01C0792379
:100C70007C939F918F9108958F9389DF8F91A0E04E
:100C8000B0E056F011968F93AF93BF9385DFBF917D
:100C9000AF918F910EF0F6CF0A2F1B2F0895AF93CF
:100CA000BF93EF93FF9338E0EEE9F0E00D910193ED
:100CB0003A95E1F7FF91EF9130E430939D003327AF
:100CC00030939A0069DF38E0BF91AF91EEE9F0E030
:100CD0000D914191041719F43A95D1F7089524DE46
:100CE0000895AF93BF930F939F938F938FB78F9375
:100CF000A0E6B0E08C9183958D938C3309F03DC0D4
:100D000088278E9311968C9183958D938C3309F05F
:100D100034C088278E9311968C9183958D9388315A
:100D200061F588278E9311968C9183958D939C9174
:100D30000EE1943089F0963079F0993069F09B306B
:100D400059F00CE1923039F411969C9111979370FF
:100D500019F4039501C00FE1801778F071F081E07C
:100D60008E9311968C9183958D938D3031F481E023
:100D70008E9311968C9183958C938F918FBF8F91C9
:100D80009F910F91BF91AF911895000F111F221FD6
:100D9000331F089500951095209530950F5F1F4FD4
:100DA0002F4F3F4F0895019110810EC00191119175
:100DB000219130810BC00191108117FF05C03FEFD9
:100DC0002FEF04C0008111272227332737FF03C0EC
:100DD000E1DF8DE28D93CF93DF93CF92DF92EF929D
:100DE000AA24BB24CC24DD24EE2440E2CAE0DD2783
:100DF00055E093E38881890F87FD9F7083FD907F85
:100E0000891B89935A95A9F7C0DFAA1CBB1CCC1C6F
:100E1000DD1CEE1C4A9551F7E894EFE0FF27829124
:100E20000ED0EB30E0F71EF068948A2D0CD08827A6
:100E30008D93EF90DF90CF90DF91CF910895982F11
:100E4000829501D0892F8F70805D26F0803309F460
:100E5000089568948D93089594E081918D939A9567
:100E6000E1F7089500276CE8719198E00695779571
:100E700077FF18F477FD08F006279A95B9F78A9559
:100E800099F70895327844533138423230207468EB
:100E900065726D6F000020594F365049522028521C
:100EA0002920323031310000204453313D31384265
:100EB00032302020202020200000204453313D31BA
:100EC000385332302831383230290000204E4F203C
:100ED00053656E736F723120212020200000202086
:100EE00020445331203D3E20445332202020000036
:100EF000204453323D3138423230202020202020FF
:100F00000000204453323D313853323028313832DA
:100F100030290000204E4F2053656E736F723220CF
:100F2000212020200000457874005B0030003A004A
:100F30005D20496E740045727244533100004300D5
:080F40004572724453320000B7
:00000001FF
